S02100006E6573742D626F6F746C6F616465722D7370692D656D333538312E73333778
S3150800000000040020490200085502000855020008AD
S31508000010A70B0901000000000101022000400008AA
S31508000020040A0000570D00080D10000828060008ED
S3150800003000000000000000000000000000000000B2
S315080000400000000000000000000000007D00000025
S315080000500000000010B501210E2000F04BF8124CEC
S315080000604020A060642000BF401EFCD108210E205D
S3150800007000F040F84FF4FA7000BF401EFCD1246827
S3150800008004210E2000F036F8A00900F0010080F0E7
S31508000090010010BD80B500F022F80448016841F05F
S315080000A01001016001BD000008B2004000BC00401C
S315080000B07047000018480068C00701D41748704701
S315080000C01748704780B5FFF7F5FF1649096801B963
S315080000D0400802BD80B5FFF7EDFF400802BD124893
S315080000E0012181604EF6BE21416000E00F480121E2
S315080000F00160704710B50FF23803820853F82220C2
S31508000100136800F0030080000F248440A34301FA1B
S3150800011000F01843106010BD1C400040001BB700DB
S3150800012000366E0120400040006000400860004034
S3150800013000B0004004B0004000B2004004B20040E5
S3150800014000B4004004B400401C48002101600121AD
S31508000150C1600161002141600221016018480168FF
S31508000160426841EA02416FF31311164A11438AB2F3
S315080001700260090C4160102101617047124800684D
S315080001800007FBD5704710480068800808E00F494B
S315080001904A685207FCD5086070470B480068400853
S315080001A000F00100704709494A68920703D50968B3
S315080001B001700020704701207047000054C80040B5
S315080001C000B200409044080040C800403CC80040C7
S315080001D080B500A8FFF7E7FF0028FAD001BD0000A8
S315080001E00A0242EA11214840C0F30311484080EA56
S315080001F0003041010206C9B2D20E41EA0221484046
S3150800020080B270470A0A4840C0B208214308C007AE
S3150800021046BF034858401846491EF7D15040704714
S315080002202083B8ED06480068202100EA010028B1BD
S315080002300448016842685FEA010D104770470000EC
S315080002402C00004000400008FFF7ECFF00F00EF815
S3150800025000F042F806E000005FEA000D70474548E6
S31508000260008870474FF4017000F09EB838B54FF219
S315080002700F04414DFFF7EEFE28B140F20520288015
S315080002806C80012032BD3D480068C00615D56888D7
S31508000290A0421ED1288840F2022188421CBF40F2A3
S315080002A00621884215D040F2011188421EBFB0F5DA
S315080002B08A7F40F2111188420BD0314C208A40F6D1
S315080002C0A721884205D12068FFF7C6FF60688047E6
S315080002D000BF002032BD000038B50446294872B672
S315080002E0016849084900016000F08AF82348006857
S315080002F0000910F001000CBF2349244902E0CD2271
S3150800030001F8012B224A9142F9D32249224A234B6A
S3150800031003E011F8015B02F8015B9A42F9D3204920
S31508000320204A002301E001F8013B9142FBD3124A1F
S3150800033053884FF20F0540F20521AB420AD11388C4
S315080003408B4205D030B1180A012818BF022801D1FE
S31508000350194601E004B90021064801804CF23C30F8
S31508000360508000F03DF94FF40170BDE8324000F0CE
S315080003701BB8000020070020000000202C000040C9
S3150800038000400008FCED00E0000000209800002076
S3150800039000040020C01200080004002010040020F9
S315080003A010040020270700200D4930220A600D4955
S315080003B00A600D490A600D4910220A60010A08BF41
S315080003C000020B4908804FF20F004880BFF35F8F89
S315080003D008480021016041600748084901607047E4
S315080003E03020004030C8004030C0004010E00040D7
S315080003F0000000201C4000400CED00E00400FA0557
S3150800040029E038B50546FFF75DFE6B49B0FBF1F408
S315080004104FF4F070B0FBF4F02D1A1E2DBCBF4FF44C
S315080004200170FFF7C1FF654807210160002141609F
S31508000430816063494FF000720A6005FB04F1C91C2C
S315080004408908491E416031BD5F48016841F00101D4
S315080004500160012141605D4851210160704700201B
S3150800046070472DE9F047814640F2DC58C246584E9F
S315080004705248584F584C534D296801291DDA022114
S31508000480618039600068C00348BF00F07CF8B8692D
S3150800049000F00300032864D02868002803D5B8694B
S315080004A040F00200B8614846FFF7D9FF5FEA000A44
S315080004B01BD12868002854D551E04FF6FF7561888E
S315080004C0A94220D102237F2244480188A01C00F0BB
S315080004D0AFF86088A84204BF02206080B869800728
S315080004E003D4B86940F00200B8610120B070608892
S315080004F03860012070700FFA8AF42046FFF781FFF2
S31508000500A0B2BDE8F087B9698907EAD50068C003D3
S3150800051048BF00F038F8B07808B14046F1E7B86847
S3150800052010F00100B968628803D10F2A08D2521C5C
S3150800053006E0890704D5217811B1032A28BF521E7F
S31508000540207092B2022A38BF022262803868618817
S315080005508842CAD1B86900F00300032801D0FFF722
S3150800056073FF0020CDE710B5044604E000F094F8C8
S315080005700620FFF774FF2046FFF773FF0028F5D122
S3150800058010BD0220EFE70D48002141608160016837
S3150800059021F0020101600E480021417008494FF020
S315080005A000720A60817801B9704780B500218170B0
S315080005B00620FFF754FF01BD90D0030010E000E0CD
S315080005C004ED00E0B81200081C400040008000401E
S315080005D022070020044000400C040020BC1200083A
S315080005E080B5FFF7CEFFFFF73AFEB0F58A7F09D14F
S315080005F0FFF7AAFDFFF7D1FD0028FBD040F2111046
S31508000600FFF7D2FEFFF746FDFFF79EFD00F006F95D
S3150800061040F20120FFF7C8FE002002BD012A08BFEC
S31508000620FFF7B5BD704700006F120008A712000853
S3150800063030B50446104683B07F2808BF0020B1F5C0
S31508000640004F1AD108237F2240F6120100A8FFF7AF
S31508000650EFFF08220FF2380100A800F021F930B99F
S3150800066008237F2240F2A27100A8FFF7E1FF0822C3
S3150800067000A9204600F0F4F837BD044D294300FBD5
S3150800068003111A46204600F0EBF837BD00000808AB
S31508000690FFFFFFFFFFFFFFFF70B506460C4C2568FE
S315080006A0FFF718FD0B49B0FBF1F070432F303021EE
S315080006B0B0FBF1F0032809D3616D41F001016165D2
S315080006C02168491B0903090B8142F9D370BD000053
S315080006D03820004090D003000A0A4840C0B20821DA
S315080006E04308C00746BF574858401846491EF7D121
S315080006F050407047F0B5044687B0E0885249534DDC
S3150800070007286ED8DFE800F00419213B666D0C4D0A
S3150800071043F2815301220021281D00F0E1F810E080
S31508000720E168206900291DBF616901606269026884
S315080007300621281D00F0E6F803E00121281D00F037
S31508000740E3F8281D00F052F94BE0E068884212D31E
S31508000750206900F2FF70C50A002608E0E06800EB91
S31508000760C621022000F040FAFFF7C0FC761CAE4214
S31508000770F4D3324601E04FF0FF3202210DE0E06883
S31508000780FF22884208D321694A0804F1140100F0BF
S3150800079049FA020008BFE268032100A800F0CFF872
S315080007A014E0E6684FF0FF35002707E0B85D2946F4
S315080007B0FFF792FF0546FFF799FC7F1C20698742E1
S315080007C0F4D32A46072100A800F0C3F800A800F0D1
S315080007D00DF906E00022042100A800F0B0F8012077
S315080007E0286007B0F0BD10B50446012000F004F9F2
S315080007F0A08828B1022804BF2046FFF77BFF08E03F
S31508000800124C0FF24C01201D00F05AF8201D00F082
S31508000810EDF8002000F0F0F8002010BD10B500F04B
S31508000820A5F8FFF763FC094C08E0FFF75FFC00F04A
S31508000830B7F908B900F0CDF800F0E8F82068002804
S31508000840F3D010BD2083B8ED002000081004002066
S315080008506E6C626C2D656D3335782D312E30320015
S31508000860814212D210185118401E491E92B2002A0F
S315080008701EBF11F8013900F80139521EF6D170472A
S3150800088011F8013B00F8013B521E92B2002AF7D13B
S315080008907047130003D00A46194600F0E9B97047B5
S315080008A010B500E0521E92B23AB110F8013B11F8A9
S315080008B0014BA342F6D0181B10BD002010BD000046
S315080008C038B50D46044621230022002100F003FA1C
S315080008D0294604F10C00BDE838401022FFF7C0BFD6
S315080008E070B515461E460A4604461923022100F02D
S315080008F0F2F9A581E6810248206170BD000000007A
S3150800090068616C6F38B51BE010B50A460446552376
S31508000910022100F0E0F90120A0814FF0006104F106
S315080009200C0041604FF400618160C1606021018262
S315080009304FF032314164FF2084F8540010BD38B5B9
S3150800094015460A4604461523022100F0C4F9E56057
S3150800095031BD38B5F4E700009348002101704FF027
S31508000960FF319248016041608160704780B5FFF7AA
S31508000970EBFB8F48016821F470410160016841F47E
S315080009808051016001BDF8B5164600240D464FF0AA
S31508000990FF37B6F5807FC8BF3C4618DC38B1321D34
S315080009A0014692B28348FFF75BFF002000E0384615
S315080009B07E49086005B100274F608E60012E7A488F
S315080009C002DB0121017002E0062202708C602046DB
S315080009D0F2BD80B54FF48072EE217748FFF759FFD4
S315080009E0BDE80840002201210020CCE7B0F902103A
S315080009F0CA1C0021401CC6E770490028086814BFB5
S31508000A0040F0800020F08000086070472DE9F04132
S31508000A10654D664EA8682A7871680024401C521EE7
S31508000A2082B04FF0FF38644F062A0BD8DFE802F091
S31508000A300B042A8190556B00FFF7A0FBFFF7C8FB54
S31508000A40AC602C70A9E03068002812D407E0594938
S31508000A50405CFFF79CFB3068AC60401C3060FFF7D9
S31508000A6092FB18B13068B1688842F0DBA868401C70
S31508000A70A8603068B1688842C0F288800220287071
S31508000A8001248AE000291BD40FE000A8FFF78BFB9E
S31508000A9070689DF80010C155401C706069689DF823
S31508000AA00000FFF7AFFB6860AC60FFF776FB20B18C
S31508000AB0B1687068091D8842E7D3A868401CA86019
S31508000AC0B1687068091D884260D302202870012425
S31508000AD069683846FFF787FE5FE000295DD1FFF7B2
S31508000AE05CFB002859D000A8FFF75DFB9DF80000C5
S31508000AF0FF2852D170689DF80010C155401C7060DF
S31508000B000720287049E0A86001293FD1FFF745FB77
S31508000B10002842D000A8FFF746FB9DF80000FE28F3
S31508000B203BD170689DF80010C155401C70600420C8
S31508000B300BE0A860FFF731FB40B37068C019FFF7F8
S31508000B4032FB7068401C706005202870AC6024E099
S31508000B50A860FFF722FBC8B17068C019FFF723FB2E
S31508000B607068401C7060F978B878AC6050EA01206B
S31508000B70B06007D0B0F5827F04D803202870C5F886
S31508000B8004800AE04446FFF724FF06E0A8680C49FB
S31508000B90884202D3FFF7E0FE44462046BDE8F681C8
S31508000BA00148007870470000140500200004002062
S31508000BB004B2004020050020200600200CB20040A8
S31508000BC0A08601002748018A40F6A772914202BF13
S31508000BD0418A4FF47F40014204D102298041C04333
S31508000BE0C00F704700207047F8B504460D461C4EE6
S31508000BF001203070FFF7E6FF18B94FF40170FFF7D0
S31508000C00D3FB1848876A294644F48070B847002100
S31508000C1031700FF2540618B9294644F40070B847E3
S31508000C20805DF2BD2DE9F041044688465600FFF77F
S31508000C30C9FF18B94FF40170FFF7B6FB0948476AB0
S31508000C400023324641462046B8470FF21C0520B914
S31508000C503346002241462046B847405DBDE8F0814C
S31508000C602607002000000808000202024B4B4647F0
S31508000C7062F30F2262F31F42401810F0030308D0F4
S31508000C80C91A1FD3DB0748BF00F8012D28BF20F873
S31508000C90022D130030B414461546103928BF20E932
S31508000CA03C00FAD8490728BF20E90C0048BF40F89D
S31508000CB0042D890028BF20F8022D48BF00F8012D11
S31508000CC030BC7047C91818BF00F8012DCB0728BFDC
S31508000CD000F8012D704710B54FF6FF6404801B1FFE
S31508000CE0438041F400418180C28010BDF8B50446B6
S31508000CF00D4616461F4607E03046A0472946FFF729
S31508000D0081FA05467F1E761CBFB2002FF4D128460D
S31508000D10F2BD38B50C46154605E0014614F8010B38
S31508000D20FFF770FA6D1EADB2002DF6D132BDF8B5DB
S31508000D3004460D4616461F463A4631462868236835
S31508000D409847040005D13A463146E868FFF7E1FFBF
S31508000D50E8602046F2BD10B5029C847203814260A9
S31508000D6001604FF0FF31C1600021017410BD2DE90B
S31508000D70F84F04468B461E469BF81B70802F28BFEB
S31508000D808027D0689D49884250D1002E4CD0B06843
S31508000D9000904FF0FF384FF000090BEB490A9AF81C
S31508000DA048500FE0FF2D16D0FFF7A0F94FF4006367
S31508000DB0E80240F0006241460098FFF797FF804638
S31508000DC0681CC5B29AF84900A842EBDA09F101098C
S31508000DD0B9F1060FE1DBDBF844006FEA0801884247
S31508000DE024D1A06800BA7A08594673689847C8B9E2
S31508000DF0E06805BAA06802BA3B464FF0FF31B06812
S31508000E00FFF774FFC04385420CD140F6A720ABF824
S31508000E101000A06800BA01220BF1100110307368A7
S31508000E20984708B1422002E0172000E04320BDE8B9
S31508000E30F28F2DE9F84F80460D469146D5F804A065
S31508000E402889ADF8000005F1140606F110070423F9
S31508000E5052464046FFF76BFF002870D1BAF80000EB
S31508000E6040BA1FFA80FBBAF8020040BA84B2E0071B
S31508000E7048BF462063D4B4F5026FC8BF4E205EDC77
S31508000E80002C5BD05FEA0B000AD04FF60441BBEB9F
S31508000E90010000F09B80FF3853D0FE3851D0ABE0FC
S31508000EA0287C08B151204AE08D2C28BF4F2046D215
S31508000EB02346321D00F0A7F8002840D1FA7E802A82
S31508000EC028BF802202F10C00844201BFB08840BAD4
S31508000ED000F47F40B0F5007F2CD1F08840BA4EF27E
S31508000EE05031884202BF388A40F6A721884202BF9D
S31508000EF0788A00F47F40B0F5807F1BD1B06800BACD
S31508000F003F49C969884215D14FF6FF70388206F104
S31508000F1010014FF0FF30FFF7FCFEF16809BAC9432C
S31508000F20884204BF387E042804D1787E0A2818BF70
S31508000F30062801D0452002E0012028740020BDE8DB
S31508000F40F28F287C002843D0042300F05BF80028A1
S31508000F50F5D1DAF8000006BA201F84B22848C0691D
S31508000F60864238BF4820EAD3A019796D884228BF3F
S31508000F704920E4D24FF6035083450DD1B9F1000F4D
S31508000F800AD031460220D9F80020904720B14A20DD
S31508000F90D5E7E01B84B2BE19002CCFD0BDF80000FF
S31508000FA08442B4BF274607463B4600F02BF8002884
S31508000FB0C5D1B9F1000FECD07A0851463046D9F8B8
S31508000FC0043098470028E4D04B20B8E7287C08B9B5
S31508000FD04120B4E7042C18BF4C20B0D104236A681A
S31508000FE000F011F80028AAD14B462A463946304661
S31508000FF001B0BDE8F04FBAE64420A0E7E320BBDE27
S315080010000000000852462946404690E670B5044658
S315080010100D4616462889C10701D4802803DA4F20D1
S3150800102070BDA87A78B9324629462046FFF701FFEF
S315080010300028F6D0172807D1286861688847172836
S3150800104002D1002070BD502070BD0000F8B50446DE
S315080010500D46164616484FF0FF310160134FFE62E3
S3150800106000207862386840F001003860FFF73EF8E3
S31508001070012C19D16DB9FFF790F878B9786AB042A2
S31508001080F4D3002EF2D038684008400038601620A5
S31508001090F2BD2846FFF787F80028EFD138684008E0
S315080010A0400038600020F2BD0120F2BD00F000408B
S315080010B000A8004038B504460D4600F009F800F0CF
S315080010C007F82A4621461820BDE83840FFF7A6BA91
S315080010D02A4621461820FFF7A1BA30B583B0044640
S315080010E0002020814AF6B43200A92078FFF7AEFF27
S315080010F008B11C203EBD9DF80000032818BF18281B
S3150800110001D118203EBD042801D117203EBD012873
S3150800111001D021203EBD002500E06D1CEDB2A1885E
S31508001120091D8D420BDA40F2DD22281900F10A0169
S315080011302078FFF78BFF0028EFD026203EBD00253C
S31508001140002006E00146EDB22819007BFFF748F8B3
S315080011506D1CA188EAB28A42F4D3A27AE37A9B1874
S31508001160FF2B01D022203EBD0B191D7BB5EB102F9E
S3150800117001D023203EBD5B7BC0B2834201D0242030
S315080011803EBDA078824207D0401EC0B2824201D13D
S3150800119027203EBD25203EBD881C20810220E080F8
S315080011A000203EBD38B504466078012804D023D314
S315080011B0032855D018D31FE02078012811D13B25E4
S315080011C04320FEF7E4FF40F2DD2200212078FFF7F6
S315080011D03DFF30B12846451EC0B20028F0D11B207D
S315080011E032BD0220607010E0FEF7F2FF00F03AF818
S315080011F0A078401CA07008E0182032BD2278A0789C
S31508001200411EC9B20620FFF709FA2046FFF765FF17
S31508001210050018BFFEF7DCFF272DEFD0A8060BD573
S315080012202278A1781520FFF7F9F9002DEDD10320D2
S31508001230FEF73EFF002032BD680603D4182D18BFFE
S315080012401C2D07D121782846FFF734FF042060704B
S31508001250284632BD172DE8D100F004F80320607047
S31508001260172032BD2278A1780620FFF7D7B9F8B53E
S3150800127004460D461646002706E0E088411CE18034
S315080012800019807A78557F1CBFB2B74209D2E08828
S3150800129021898842F1D32046FFF784FF0028ECD045
S315080012A0F2BD0020F2BD10B504462046FFF77AFFCE
S315080012B00028FAD010BD000000366E01EE080000C6
S315080012C0FFFFFFFFFFFFFFFFFFFFFFFF0100FFFF1D
S70508000249A7
